:100000000C9466000C948E000C948E000C944106A7
:100010000C946B060C9495060C948E000C94650E53
:100020000C948E000C948E000C948E000C9403089B
:100030000C948E000C948E000C948E000C948E0008
:100040000C94C1080C948E000C94BA0B0C940C0CFC
:100050000C948E000C948E000C948E000C948E00E8
:100060000C9446040C948E0000000000240027002D
:100070002A0000000000250028002B0000000000DE
:1000800023002600290004040404040404040202DA
:100090000202020203030303030301020408102007
:1000A0004080010204081020010204081020000012
:1000B0000007000201000003040600000000000029
:1000C00000000200CC00B3037B0DC50011241FBE4D
:1000D000CFEFD8E0DEBFCDBF11E0A0E0B1E0EEE0B1
:1000E000FBE202C005900D92A234B107D9F713E0EC
:1000F000A2E4B1E001C01D92A23EB107E1F710E019
:10010000CAECD0E004C02297FE010E947615C43CE0
:10011000D107C9F70E94D20D0C947A150C940000F7
:10012000FB01DC0102C001900D9241505040D8F714
:100130000895FB01DC0101900D920020E1F7089584
:10014000CF93DF9381309105A1F46F5F7F4FD1F49E
:10015000C2E4D1E0CE010E94BF06239681E0CA35F9
:10016000D807C1F780E691E060E071E00E94891154
:1001700009C0892B39F46F5F7F4F21F480E691E04D
:100180000E94A211DF91CF91089580E090E06FEF7F
:100190007FEF0E94A000089581E090E06FEF7FEF75
:1001A0000E94A00008951F9312E0812F61E00E9439
:1001B000370A812F60E00E94760A1F5F1C30A9F782
:1001C0001F910895EF92FF920F931F93DF93CF93A8
:1001D00000D00F92CDB7DEB720916701222319F02E
:1001E0000091A20102C000916E01602F70E0813287
:1001F000910509F45DC0823291053CF48E31910580
:1002000059F0809709F0A7C018C08232910539F1E2
:10021000C29709F0A0C08DC0802F61E00E94370A0C
:1002200080916701882319F06091A30102C0609159
:100230006F01802F0E94760A8EC0802F61E00E949D
:10024000370A80916701882319F06091A30102C0E9
:1002500060916F01802F70E00E94D7097CC0802FD1
:1002600061E00E94370A80916701882349F020915C
:10027000A3019091A4014091A5018091A60108C01D
:1002800020916F01909170014091710180917201F4
:10029000792F60E0620F711D382F20E0240F311D8F
:1002A000442737FD4095542F802F0E94C10E53C024
:1002B000222319F08091A30102C080916F01E82EE2
:1002C000FF2485EBE816F10408F045C0E4EDF1E009
:1002D00080E090E0208131812617370789F0232BB9
:1002E00041F4FC01EE0FFF1FEC52FE4F718360835F
:1002F00007C0019632968830910561F780E090E062
:10030000FC01EE0FFF1FE80FF91FDE011196EE5BF7
:10031000FE4F83E001900D928150E1F78E010F5F57
:100320001F4FC8010E94FC07C801B7010E941507B2
:1003300012C00E9409090E94571420E030E04AE7E9
:1003400054E40E94BE136093E5017093E60180932C
:10035000E7019093E8010F900F900F90CF91DF91FC
:100360001F910F91FF90EF9008951092660187EA18
:1003700093E00E94CE0C181619065CF481E080937D
:1003800066011092670187EA93E00E94020D809354
:10039000D3010895682F87EA93E00E943B0D0895EA
:1003A000EF92FF920F931F937B018C0183E00E94D9
:1003B000CA01C801B7010E94261470935F016093BF
:1003C0005E0180915E010E94CA0180915F010E94DE
:1003D000CA011F910F91FF90EF900895EF92FF9245
:1003E0000F931F937B018C0182E00E94CA01E0926F
:1003F0005A01F0925B0100935C0110935D018091C2
:100400005A010E94CA0180915B010E94CA01809139
:100410005C010E94CA0180915D010E94CA011F9186
:100420000F91FF90EF900895DF92EF92FF920F935C
:100430001F9320916701222319F0D090A20102C0DE
:10044000D0906E018432910509F459C0853291052E
:100450003CF48E31910559F04F9709F092C00FC0CE
:100460008532910519F1C29709F08BC080C08D2D9E
:1004700060E00E94370A8D2D0E94CA0A0EC0ED2D41
:10048000F0E0EE0FFF1FE65FFE4F1081812F60E06E
:100490000E94370A812F0E94B509AA2797FDA095CF
:1004A000BA2FBC01CD010E94591469C0222319F052
:1004B0008091A30102C080916F0180935E0122238D
:1004C00019F08091A40102C08091700180935F01B6
:1004D000E0905E01F0905F018D2D60E00E94370A90
:1004E0000027F7FC0095102F8D2D61E0A8019701E2
:1004F0000E941D0B0E9457140E94D00142C022236B
:1005000029F01091A201E090A30104C010916E01A6
:10051000E0906F01812F61E00E94370A812F60E037
:100520000E94760A82E090E00E947009812F61E0CB
:100530000E94760A8AE090E00E947009812F60E0B4
:100540000E94760A8E2D60E00E94370A8E2D61E0AF
:1005500020E335E740E050E00E941D0B0E94571455
:1005600020E030E048E652E40E94BE1308C06091EB
:10057000E9017091EA018091EB019091EC010E94F8
:10058000EE011F910F91FF90EF90DF9008958FEF94
:100590000E94CA0185E50E94CA01089587EA93E096
:1005A0000E940D0E08958FEF0E94CA0185E50E94FA
:1005B000CA010E94CE0208950F931F931092D20198
:1005C00080916701882349F090919E0100919F01DD
:1005D0008091A0011091A10108C090916A01009141
:1005E0006B0180916C0110916D01923019F40E94A1
:1005F000D3001EC08230B1F0833018F48130C1F4D2
:1006000005C0843099F0853099F410C00E94C7026B
:10061000802F0E94CA01812F90E00E9414020E9444
:10062000CE0206C0812F90E00E94E2000E94D30219
:100630001F910F9108950E94B50180916601882352
:1006400009F44FC02091D301253571F48091D20176
:10065000882351F48091E4018F3F31F581E080934C
:10066000D0018093D20120C02093E4018091D20177
:100670008823D1F09091D001923019F42093D101C8
:1006800007C0933028F08091D10181508093D1012F
:10069000E92FF0E080916701882319F0E456FE4FBE
:1006A00002C0E859FE4F20838091D0018F5F809374
:1006B000D001843320F01092D0011092D2018091A9
:1006C000D201882371F08091D101882351F4809167
:1006D000D001843030F01092D2010E94DC021092DE
:1006E000D00108950E94D30087EA93E040E056E9E4
:1006F00060E070E00E94470C64E670E080E090E00B
:100700000E941709089520910E0230E080910D0299
:10071000281B3109C901089540910D0280910E02F4
:10072000481718F02FEF3FEF0AC0E42FF0E0E35135
:10073000FE4F8081282F30E04F5F40930D02C901AA
:100740000895E0910D0280910E02E81718F0EFEF86
:10075000FFEF06C0F0E0E351FE4F8081E82FF0E0AC
:10076000CF0108950895109235021092340288EE58
:1007700093E0A0E0B0E08093360290933702A0931C
:100780003802B093390286E291E09093330280936D
:1007900032020895CF92DF92EF92FF920F931F9350
:1007A000CF93DF937C016B018A0180913102882312
:1007B000A1F0C0E0D0E00DC0D701ED91FC91D601D1
:1007C000AC0FBD1F0190F081E02DC7016C91099520
:1007D0002196C017D10780F304C0CB01642F0E947B
:1007E0002B04C801DF91CF911F910F91FF90EF90E3
:1007F000DF90CF900895DF93CF930F92CDB7DEB700
:10080000FC016983809131028823C9F08091300214
:10081000803238F081E090E09383828320E030E002
:1008200015C080912F02E82FF0E0E15FFD4F998124
:1008300090838F5F80932F028093300205C0CE019A
:10084000019661E00E942B0421E030E0C9010F9085
:10085000CF91DF910895482F613210F081E0089523
:1008600080913E02843011F082E008956093890205
:10087000A8E6B2E0842F9C01F90102C081918D931A
:100880008E2F841B8617D0F380E008951F920F925D
:100890000FB60F9211242F933F934F935F936F9353
:1008A0007F938F939F93AF93BF93EF93FF93809129
:1008B000B90090E0887F90708036910509F4F2C00D
:1008C00081369105CCF58832910509F47BC08932D7
:1008D0009105B4F48031910509F46FC0813191051F
:1008E0003CF4009709F447C1089709F04FC165C06F
:1008F0008831910509F466C0809709F047C182C02C
:100900008034910509F4A4C08134910544F4803306
:10091000910509F482C0C89709F038C189C08035B3
:10092000910509F489C08835910509F496C0883489
:10093000910509F02BC1AEC08839910509F413C1A6
:1009400089399105ECF48837910509F4ABC08937F2
:1009500091054CF48836910509F4A4C080379105BF
:1009600009F014C19FC08838910509F4FCC0803992
:10097000910509F49DC08038910509F007C198C020
:10098000803B910509F4C6C0813B91054CF4803A47
:10099000910509F49FC0883A910509F0F7C0BAC0E3
:1009A000803C910509F4E3C0883C910509F4DFC05F
:1009B000883B910509F0EAC0C2C080913F02809354
:1009C000BB00CFC09091660280916702981768F4CF
:1009D00090916602E92FF0E0EA5BFD4F8081809301
:1009E000BB009F5F90936602BCC080914002882349
:1009F00009F44BC085ED8093BC008091BC0084FD60
:100A0000FCCFC2C080E28093AB0285ED8093BC0036
:100A10008091BC0084FDFCCFB7C080E38093AB0223
:100A200085ED8093BC008091BC0084FDFCCFACC000
:100A300088E38093AB029BC0809166029091BB00DB
:100A4000E82FF0E0EA5BFD4F90838F5F80936602B2
:100A5000909166028091670282C0809166029091B7
:100A6000BB00E82FF0E0EA5BFD4F90838F5F80933F
:100A7000660280914002882341F085ED8093BC009E
:100A80008091BC0084FDFCCF7FC081E08093410257
:100A900084EA6EC085ED8093BC008091BC0084FD2B
:100AA000FCCF72C083E080933E021092AA0259C02C
:100AB0008091AA02803208F056C08091AA029091DB
:100AC000BB00E82FF0E0E657FD4F90838F5F8093E7
:100AD000AA0247C08091AA02803230F4E091AA02B3
:100AE000F0E0E657FD4F108285ED8093BC008091C9
:100AF000BC0084FDFCCF10923E026091AA02E091FE
:100B00004402F09145028AE892E070E00995109263
:100B1000AA022DC084E080933E02109288021092B7
:100B20008902E0914202F091430209958091890285
:100B3000882329F481E080938902109268029091C1
:100B40008802E92FF0E0E859FD4F80818093BB00D7
:100B50009F5F9093880290918802809189029817F4
:100B600010F485EC01C085E88093BC000FC085ECD3
:100B70008093BC0009C01092AB0285ED8093BC004D
:100B80008091BC0084FDFCCF10923E02FF91EF915A
:100B9000BF91AF919F918F917F916F915F914F9195
:100BA0003F912F910F900FBE0F901F9018950F93AC
:100BB0001F93CF93DF93FC01738D76957170A6859B
:100BC000B7859585772329F08C91892309F454C042
:100BD00004C08C91892309F04FC08389948920E057
:100BE00001972FEF8F3F9207D9F7C589D689A68540
:100BF000B785158560E031E040E050E000E0CE01CF
:100C0000202F01972FEF8F3F9207D9F78C918123E7
:100C100011F0632B03C0832F80956823330F4F5F40
:100C20005F4F4830510559F78789908D20E0019733
:100C30002FEF8F3F9207D9F7711160958091EE02E7
:100C40002091EF0290E001968F73907030E0821750
:100C5000930779F0E091EE02F0E0E255FD4F6083FA
:100C60008091EE0290E001968F7390708093EE0277
:100C700003C0838D8160838FDF91CF911F910F918E
:100C800008951F920F920FB60F9211242F933F9346
:100C90004F935F936F937F938F939F93AF93BF9384
:100CA000EF93FF938091AC029091AD02009711F009
:100CB0000E94D705FF91EF91BF91AF919F918F91C6
:100CC0007F916F915F914F913F912F910F900FBE48
:100CD0000F901F9018951F920F920FB60F9211242C
:100CE0002F933F934F935F936F937F938F939F9334
:100CF000AF93BF93EF93FF938091AC029091AD02BD
:100D0000009711F00E94D705FF91EF91BF91AF912D
:100D10009F918F917F916F915F914F913F912F9113
:100D20000F900FBE0F901F9018951F920F920FB645
:100D30000F9211242F933F934F935F936F937F9361
:100D40008F939F93AF93BF93EF93FF938091AC02E8
:100D50009091AD02009711F00E94D705FF91EF919D
:100D6000BF91AF919F918F917F916F915F914F91C3
:100D70003F912F910F900FBE0F901F901895FC017F
:100D80008091F0028C3090F480838F5F8093F0022A
:100D9000815090E0FC01EE0FFF1FE80FF91FEF50AC
:100DA000FD4F88EB9BE09283818308958FEF8083D2
:100DB0000895FC0120812C30B8F58181992787FDA9
:100DC000909548E850E0481B590B440F551F440FBD
:100DD000551F6417750784F08281992787FD9095C8
:100DE00048E552E0481B590B440F551F440F551F4F
:100DF000641775070CF4AB0142505040CA01AA2792
:100E000097FDA095BA2F880F991FAA1FBB1F4FB738
:100E1000F89430E0F901EE0FFF1FE20FF31FEF50DF
:100E2000FD4F928381834FBF0895AF92BF92CF92BF
:100E3000DF92EF92FF920F931F93CF93DF93EC011A
:100E40009B0182E0603278070CF048C077FF03C056
:100E500020E030E005C0653B710514F024EB30E084
:100E600000D000D0B901882777FD8095982F29817F
:100E7000332727FD3095E8E8AE2EB12CA21AB30A2D
:100E8000AA0CBB1CAA0CBB1CCC24B7FCC094DC2C49
:100E9000EA81FF27E7FDF09528E532E02E1B3F0BA6
:100EA000220F331F220F331F442737FD4095542F45
:100EB000EDB7FEB7218332834383548320E030E0D3
:100EC00040E050E004EBE02EF12C012D112D0E94AA
:100ED000D7109B010F900F900F900F90CE01B9018A
:100EE0000E94D906DF91CF911F910F91FF90EF9053
:100EF000DF90CF90BF90AF900895CF92DF92EF92A6
:100F0000FF921F93CF93DF93EC01162F7A016901B3
:100F100088818C3008F064C0862F61E00E94370A17
:100F2000888190E0FC01EE0FFF1FE80FF91FEF50E2
:100F3000FD4F1F738081807C812B808380E292E053
:100F40008E199F0964E070E00E941015698380E6A5
:100F500099E08C199D0964E070E00E9410156A8385
:100F6000A8818A2F6CE00E940415682F70E0AB0105
:100F7000440F551F460F571F440F551F440F551F51
:100F800020E030E0C901840F951FFC01EE0FFF1F28
:100F9000E80FF91FEF50FD4F808186FD15C02F5FD0
:100FA0003F4F2C30310571F724C01092800082E051
:100FB000809381001092850010928400B19A8091F4
:100FC0006F00826080936F008A2F90E0FC01EE0F2B
:100FD000FF1FE80FF91FEF50FD4F80818064808371
:100FE0008881DF91CF911F91FF90EF90DF90CF909C
:100FF0000895672BD1F2E8CF40E252E020E639E0D5
:101000000E947D0708951F920F920FB60F92112430
:101010002F933F934F935F936F937F938F939F9300
:10102000AF93BF93EF93FF938091150387FF05C0A4
:1010300010928500109284002BC020911503332755
:1010400027FD30958091F00290E02817390704F5CC
:1010500080911503992787FD9095FC01EE0FFF1FE6
:10106000E80FF91FEF50FD4F808186FF11C080917E
:101070001503992787FD9095FC01EE0FFF1FE80FE0
:10108000F91FEF50FD4F80818F7360E00E94760A58
:10109000809115038F5F80931503209115033327EB
:1010A00027FD30958091F00290E0281739070CF069
:1010B0004EC0809115038C300CF049C02091840003
:1010C0003091850080911503992787FD9095FC014B
:1010D000EE0FFF1FE80FF91FEF50FD4F8181928146
:1010E000280F391F309389002093880080911503C1
:1010F000992787FD9095FC01EE0FFF1FE80FF91F60
:10110000EF50FD4F808186FF2BC0809115039927FA
:1011100087FD9095FC01EE0FFF1FE80FF91FEF50C0
:10112000FD4F80818F7361E00E94760A19C080E4D0
:101130009CE905C08091840090918500049690936D
:101140008900809388008FEF8093150309C08091F8
:10115000840090918500049680549C4940F3EACF26
:10116000FF91EF91BF91AF919F918F917F916F917F
:101170005F914F913F912F910F900FBE0F901F9055
:1011800018951F920F920FB60F9211242F933F9331
:101190008F939F93AF93BF9380911A0390911B03FA
:1011A000A0911C03B0911D0330911E030196A11D57
:1011B000B11D232F2D5F2D3720F02D570196A11D36
:1011C000B11D20931E0380931A0390931B03A093D9
:1011D0001C03B0931D038091160390911703A091F7
:1011E0001803B09119030196A11DB11D8093160338
:1011F00090931703A0931803B0931903BF91AF9175
:101200009F918F913F912F910F900FBE0F901F9044
:1012100018958FB7F89420911A0330911B034091D1
:101220001C0350911D038FBFB901CA0108959B0192
:10123000AC017FB7F8948091160390911703A091A9
:101240001803B091190366B5A89B05C06F3F19F04C
:101250000196A11DB11D7FBFBA2FA92F982F8827F6
:10126000860F911DA11DB11D62E0880F991FAA1F55
:10127000BB1F6A95D1F7BC012DC0FFB7F8948091D0
:10128000160390911703A0911803B0911903E6B5C6
:10129000A89B05C0EF3F19F00196A11DB11DFFBF2E
:1012A000BA2FA92F982F88278E0F911DA11DB11D30
:1012B000E2E0880F991FAA1FBB1FEA95D1F7861B92
:1012C000970B885E9340C8F2215030404040504018
:1012D00068517C4F211531054105510571F608957E
:1012E000019739F0880F991F880F991F029701976E
:1012F000F1F70895789484B5826084BD84B58160E7
:1013000084BD85B5826085BD85B5816085BDEEE60D
:10131000F0E0808181608083E1E8F0E010828081EC
:1013200082608083808181608083E0E8F0E080815A
:1013300081608083E1EBF0E0808184608083E0EB7A
:10134000F0E0808181608083EAE7F0E08081846062
:1013500080838081826080838081816080838081BE
:10136000806880831092C1000895982F8E3008F015
:101370009E50977080911A018295880F880F807C0B
:10138000892B80937C0080917A00806480937A001E
:1013900080917A0086FDFCCF209178004091790001
:1013A000942F80E030E0282B392BC90108951F933A
:1013B000CF93DF93182FEB0161E00E94370A20974B
:1013C00009F44AC0CF3FD10509F449C0E12FF0E04C
:1013D000E255FF4F84918330C1F0843028F481308E
:1013E00051F08230B1F50CC0863019F1873049F1E7
:1013F000843079F514C084B5806884BDC7BD33C01E
:1014000084B5806284BDC8BD2EC080918000806894
:1014100080938000D0938900C093880024C080917D
:101420008000806280938000D0938B00C0938A00FC
:101430001AC08091B00080688093B000C093B30060
:1014400012C08091B00080628093B000C093B4005D
:101450000AC0C038D1051CF4812F60E002C0812F82
:1014600061E00E94760ADF91CF911F910895CF939A
:10147000DF93482F50E0CA0186569F4FFC013491FC
:101480004A575F4FFA018491882369F190E0880FF1
:10149000991FFC01E859FF4FA591B491FC01EE584A
:1014A000FF4FC591D491662351F42FB7F8948C91D6
:1014B000932F909589238C93888189230BC0623068
:1014C00061F42FB7F8948C91932F909589238C9386
:1014D0008881832B88832FBF06C09FB7F8948C9197
:1014E000832B8C939FBFDF91CF910895482F50E0BD
:1014F000CA0182559F4FFC012491CA0186569F4F15
:10150000FC0194914A575F4FFA013491332309F457
:1015100040C0222351F1233071F0243028F42130CF
:10152000A1F0223011F514C02630B1F02730C1F0FF
:101530002430D9F404C0809180008F7703C080915B
:1015400080008F7D8093800010C084B58F7702C0AB
:1015500084B58F7D84BD09C08091B0008F7703C0B2
:101560008091B0008F7D8093B000E32FF0E0EE0F0C
:10157000FF1FEE58FF4FA591B4912FB7F894662343
:1015800021F48C919095892302C08C91892B8C93A6
:101590002FBF0895682F70E0CB0182559F4FFC014B
:1015A0002491CB0186569F4FFC0144916A577F4F8F
:1015B000FB019491992319F420E030E03CC02223F0
:1015C00051F1233071F0243028F42130A1F0223081
:1015D00011F514C02630B1F02730C1F02430D9F411
:1015E00004C0809180008F7703C0809180008F7D40
:1015F0008093800010C084B58F7702C084B58F7D42
:1016000084BD09C08091B0008F7703C08091B00085
:101610008F7D8093B000892F90E0880F991F8458A8
:101620009F4FFC01A591B4918C9120E030E0842380
:1016300011F021E030E0C90108958F929F92AF929E
:10164000BF92CF92DF92EF92FF920F931F93CF93AF
:10165000DF93A82FB0E0CD0186569F4FFC01849008
:10166000AA57BF4FFD018491662311F4992401C04C
:10167000982C6FEFA62E6FEFB62E6FEFC62E6FE091
:10168000D62EA222B322C422D522682F70E0660F84
:10169000771F64587F4FEE24FF248701FB01A5913B
:1016A000B4910BC0EA14FB040C051D0509F44EC0EF
:1016B0000894E11CF11C011D111D8C9188218915D4
:1016C00089F30CC0EA14FB040C051D0509F43EC0A7
:1016D0000894E11CF11C011D111D03C0FB01A59123
:1016E000B4918C918821891569F720E030E040E0C1
:1016F00050E0FB01C591D4910FC0DA01C9018E0DF4
:101700009F1DA01FB11F8A159B05AC05BD05F1F0FB
:101710002F5F3F4F4F4F5F4F88818821891569F3B5
:10172000CA01B90125E130E040E050E00E94E51433
:101730009B01AC01205F3F4F4F4F5F4F84E05695B8
:101740004795379527958A95D1F704C020E030E07A
:1017500040E050E0B901CA01DF91CF911F910F9194
:10176000FF90EF90DF90CF90BF90AF909F908F90C1
:10177000089508951F920F920FB60F9211242F9380
:101780003F934F938F939F93EF93FF938091C0006C
:1017900082FD1DC04091C60020915F03309160031F
:1017A0002F5F3F4F2F7330708091610390916203E0
:1017B0002817390771F0E0915F03F0916003E15E53
:1017C000FC4F40833093600320935F0302C08091FD
:1017D000C600FF91EF919F918F914F913F912F9173
:1017E0000F900FBE0F901F901895E091B303F091EA
:1017F000B403E05CFF4F8191919120813181805C45
:101800009F4F821B930B60E470E00E941015892BA0
:1018100011F00E94B90B08951F920F920FB60F920C
:1018200011242F933F938F939F93EF93FF932091D6
:10183000A3033091A4038091A5039091A6032817D8
:10184000390731F48091C1008F7D8093C10014C0AD
:10185000E091A503F091A603ED59FC4F2081809102
:10186000A5039091A60301968F7390709093A603A1
:101870008093A5032093C600FF91EF919F918F91D4
:101880003F912F910F900FBE0F901F901895AF9220
:10189000BF92DF92EF92FF920F931F93CF93DF934C
:1018A000EC017A018B01DD24403081EE580780E0A5
:1018B000680780E0780711F0DD24D39491E0A92E29
:1018C000B12CEC89FD89DD2069F0C50108A002C0BA
:1018D000880F991F0A94E2F7808360E079E08DE336
:1018E00090E005C0108260E874E88EE190E0A80105
:1018F00097010E942315215030404040504056959A
:1019000047953795279580E12030380720F0DD2076
:1019100011F0DD24D6CFE889F9893083EA89FB8983
:10192000208319A2EE89FF89408121E030E0C901BE
:101930000C8C02C0880F991F0A94E2F7482B408351
:10194000EE89FF894081C9010D8C02C0880F991F63
:101950000A94E2F7482B4083EE89FF894081C90150
:101960000E8C02C0880F991F0A94E2F7482B40831F
:10197000EE89FF8980810F8C02C0220F331F0A94E9
:10198000E2F7209528232083DF91CF911F910F91BB
:10199000FF90EF90DF90BF90AF900895DC011C9610
:1019A000ED91FC911D97E05CFF4F81919191208119
:1019B0003181805C9F4F821B930B60E470E00E943A
:1019C00010150895DC011C96ED91FC911D97E05CCB
:1019D000FF4F20813181E054F040DF01AE5BBF4F0B
:1019E0008D919C9111972817390719F42FEF3FEF2C
:1019F00007C08D919C91E80FF91F8081282F30E05E
:101A0000C9010895DC011C96ED91FC911D97E05CE5
:101A1000FF4F20813181E054F040DF01AE5BBF4FCA
:101A20008D919C9111972817390719F42FEF3FEFEB
:101A300010C08D919C911197E80FF91F20818D9115
:101A40009C91119701968F73907011969C938E9331
:101A500030E0C9010895DC0191968C91919788231B
:101A600039F05496ED91FC915597808186FFF9CF1E
:101A700091961C920895CF93DF93EC01EE85FF853C
:101A8000E05CFF4F20813181E054F0402F5F3F4FF9
:101A90002F733070DF01AE5BBF4F8D919C9111971A
:101AA00028173907D1F3E05CFF4F80819181E05422
:101AB000F040E80FF91F6083EE85FF85E05CFF4F83
:101AC00031832083EE89FF89208181E090E00F8CB3
:101AD00002C0880F991F0A94E2F7282B208381E027
:101AE00089A3EC89FD8980818064808381E090E016
:101AF000DF91CF9108951092AA031092A90388EE66
:101B000093E0A0E0B0E08093AB039093AC03A0938C
:101B1000AD03B093AE0386E391E09093A803809366
:101B2000A7038FE193E09093B4038093B30383E61C
:101B300093E09093B6038093B50385EC90E0909387
:101B4000B8038093B70384EC90E09093BA0380933A
:101B5000B90380EC90E09093BC038093BB0381ECCD
:101B600090E09093BE038093BD0382EC90E090934D
:101B7000C0038093BF0386EC90E09093C2038093F0
:101B8000C10384E08093C30383E08093C40387E0B0
:101B90008093C50385E08093C60381E08093C703EB
:101BA00008950895CF93DF930E947A090E94D10D82
:101BB0000E947203C5EFDBE00E941B032097E1F354
:101BC0000E94F50BF9CFCF92DF92EF92FF920F9325
:101BD0001F93CF93DF937C016B018A01C0E0D0E0BB
:101BE0000FC0D6016D916D01D701ED91FC9101906F
:101BF000F081E02DC7010995C80FD91F0150104091
:101C00000115110571F7CE01DF91CF911F910F9151
:101C1000FF90EF90DF90CF900895EF92FF920F9397
:101C20001F938C01DC01ED91FC910190F081E02D7E
:101C30006DE009957C01D801ED91FC910190F08156
:101C4000E02DC8016AE009959C012E0D3F1DC901D8
:101C50001F910F91FF90EF900895813041F08130F6
:101C600018F08230D1F409C010926E00089580916E
:101C70006F008D7F80936F000895809170008D7F3D
:101C80008093700081E08093B0008091B100887FE4
:101C900084608093B1001092B30008951F93182FB1
:101CA00080911B01811711F09FEF06C0E2ECF0E07C
:101CB00094918FEF80931B01892F0E942D0E812F0D
:101CC00060E00E94760A1F9108951F920F920FB64E
:101CD0000F9211242F933F934F935F936F937F93B2
:101CE0008F939F93AF93BF93EF93FF938091D7030D
:101CF0009091D803A091D903B091DA030097A10580
:101D0000B10551F1E091DB03F091DC03808190910A
:101D1000DD03892780838091D7039091D803A09118
:101D2000D903B091DA03181619061A061B06C4F473
:101D30008091D7039091D803A091D903B091DA0391
:101D40000197A109B1098093D7039093D803A09379
:101D5000D903B093DA0304C080911B010E944E0E98
:101D6000FF91EF91BF91AF919F918F917F916F9173
:101D70005F914F913F912F910F900FBE0F901F9049
:101D800018952F923F925F926F927F928F929F92BF
:101D9000AF92BF92CF92DF92EF92FF920F931F9379
:101DA000DF93CF9300D000D0CDB7DEB7A82F1B01B3
:101DB00029833A834B835C8380911B018A1721F42A
:101DC000E2ECF0E0549082C08F3F09F0DAC1A093BA
:101DD0001B01E2ECF0E054902FEF521609F4D1C150
:101DE00081E0581639F192E0591609F449C055209E
:101DF00009F06CC014BC15BC84B5826084BD85B587
:101E0000816085BD2A2F30E0F901EA57FF4FE49148
:101E1000F0E0EE0FFF1FEE58FF4F859194919093E5
:101E2000CE038093CD0326563F4FF90184918093D2
:101E3000CF034EC0109280001092810080918100EB
:101E4000886080938100809181008160809381000F
:101E50002A2F30E0F901EA57FF4FE491F0E0EE0F4E
:101E6000FF1FEE58FF4F859194919093D503809377
:101E7000D40326563F4FF90184918093D60328C09E
:101E80001092B0001092B1008091B00082608093F7
:101E9000B0008091B10081608093B1002A2F30E0C2
:101EA000F901EA57FF4FE491F0E0EE0FFF1FEE5803
:101EB000FF4F859194919093DC038093DB0326562A
:101EC0003F4FF90184918093DD0302C057FC59C153
:101ED0008A2F61E00E94370A552021F0F2E05F1658
:101EE00009F0BEC031018824992460E072E18AE7DC
:101EF00090E0A40193010E94451559016A018601F1
:101F000075010894E108F108010911092FEFE216A3
:101F1000F1040105110509F008F499C060E472E4C8
:101F20008FE090E0A40193010E94451579018A0198
:101F30000894E108F1080109110982E05816C1F47A
:101F40009FEFE916F1040105110509F008F484C0BA
:101F500060E970ED83E090E0A40193010E944515D3
:101F600079018A010894E108F1080109110983E067
:101F7000AFEFEA16F1040105110509F008F468C095
:101F800068E478EE81E090E0A40193010E94451599
:101F900079018A010894E108F10801091109552025
:101FA00011F483E01DC0B2E05B1611F084E018C0AC
:101FB000EFEFEE16F1040105110509F008F4DFC09A
:101FC00064E274EF80E090E0A40193010E94451563
:101FD00079018A010894E108F1080109110985E0F5
:101FE000FFEFEF16F1040105110591F188F162E1AF
:101FF0007AE780E090E0A40193010E944515790101
:102000008A010894E108F10801091109552011F02D
:1020100086E001C084E02FEFE216F104010511050E
:10202000B9F0B0F0C601B50120E034E040E050E086
:102030000E94451579018A010894E108F108010917
:102040001109552011F087E008C085E003C081E048
:10205000552019F485BD3AC082E08093B10036C0A6
:102060005101CC24DD2460E072E18AE790E0A60112
:1020700095010E94451579018A010894E108F1084B
:102080000109110980E0E81680E0F80681E0080700
:1020900080E0180710F491E010C068E478EE81E069
:1020A00090E0A60195010E94451579018A010894E6
:1020B000E108F1080109110993E0A1E05A1631F491
:1020C00080918100887F982B9093810089819A81EB
:1020D000AB81BC810097A105B10529F48FEF9FEF7B
:1020E000AFEFBFEF13C0220C331CB10180E090E0D2
:1020F00029813A814B815C810E94E51428EE33E00E
:1021000040E050E00E942315C901DA01E1E05E16CB
:10211000A1F0F2E05F1619F1552099F5E7BC809324
:10212000C9039093CA03A093CB03B093CC038091CF
:102130006E00826080936E0024C0F0928900E0926D
:1021400088008093D0039093D103A093D203B093DF
:10215000D30380916F00826080936F0012C0E09281
:10216000B3008093D7039093D803A093D903B0937F
:10217000DA038091700082608093700002C084E076
:102180006CCF0F900F900F900F90CF91DF911F9118
:102190000F91FF90EF90DF90CF90BF90AF909F9006
:1021A0008F907F906F905F903F902F9008952F9227
:1021B0003F924F925F926F927F928F929F92AF92D7
:1021C000BF92CF92DF92EF92FF920F931F93DF9314
:1021D000CF93CDB7DEB73B014C0119012A016D89C0
:1021E0007E898F89988D6A197B098C099D09621AED
:1021F000730A840A950AA40193010E94E514E21867
:10220000F30804091509A80197010E9445152A0D34
:102210003B1D4C1D5D1DB901CA01CF91DF911F917E
:102220000F91FF90EF90DF90CF90BF90AF909F9075
:102230008F907F906F905F904F903F902F90089578
:102240000F931F93CF93DF93EC018B016F5F7F4F51
:10225000888199810E94DD12009711F480E005C009
:10226000998388831B830A8381E0DF91CF911F913B
:102270000F910895CF93DF93EC0188819981892B89
:1022800029F08A819B818617970760F4CE010E940E
:102290002011882341F08C819D81892B19F4E881DC
:1022A000F981108281E0DF91CF910895CF93DF9380
:1022B000EC0188819981009711F00E9445121982E2
:1022C00018821D821C821B821A82DF91CF91089591
:1022D000EF92FF920F931F93CF93DF93EC017B015B
:1022E0008A01BA010E943A11882321F4CE010E948A
:1022F000561107C01D830C8388819981B7010E9404
:102300009900CE01DF91CF911F910F91FF90EF9037
:102310000895CF93DF93EC01198218821B821A82F1
:102320001D821C826115710551F0DB010D900020AA
:10233000E9F71197A61BB70BAD010E946811DF9159
:10234000CF910895FC01808191810E9445120895EA
:102350000F931F93CF93DF93BC018230910510F44C
:1023600062E070E0E091E003F091E103A0E0B0E012
:1023700040E050E024C08081918186179707D0F01B
:102380008617970771F482819381109729F013962D
:102390009C938E9312972CC09093E1038093E0035B
:1023A00027C04115510519F08417950718F4EF015E
:1023B0008D01AC01DF01828193819C01F90130978D
:1023C000D1F641155105F9F0CA01861B970B8430EF
:1023D000910580F48A819B810115110521F0F80196
:1023E0009383828304C09093E1038093E003FE0112
:1023F000329645C0FE01E80FF91F61937193029771
:10240000998388833CC08091DE039091DF03892B00
:1024100041F480911E0190911F019093DF038093FE
:10242000DE0340912001509121014115510541F4F5
:102430004DB75EB780911C0190911D01481B590B4F
:102440002091DE033091DF0324173507B0F4CA0171
:10245000821B930B8617970780F0AB014E5F5F4F8F
:102460008417950750F0420F531F5093DF0340939A
:10247000DE03F9016193719302C0E0E0F0E0CF0167
:10248000DF91CF911F910F910895CF93DF939C011E
:10249000009709F48FC0EC0122971B821A82609189
:1024A000E0037091E1036115710581F488819981E0
:1024B000820F931F2091DE033091DF032817390725
:1024C00039F5D093DF03C093DE0374C0DB0140E035
:1024D00050E0AC17BD0708F1BB83AA83FE01219130
:1024E0003191E20FF31FAE17BF0779F48D919C91E4
:1024F0001197280F391F2E5F3F4F3983288312967B
:102500008D919C9113979B838A834115510571F49A
:10251000D093E103C093E0034DC012968D919C913E
:102520001397AD01009711F0DC01D3CFDA011396B8
:10253000DC93CE931297FA0121913191E20FF31FB0
:10254000CE17DF0769F488819981280F391F2E5F24
:102550003F4FFA01318320838A819B819383828359
:10256000E0E0F0E0DB0112968D919C9113970097CB
:1025700019F0BC01FD01F6CFAB014E5F5F4FDB01EF
:102580008D919C91840F951F2091DE033091DF0384
:102590002817390779F4309729F41092E103109243
:1025A000E00302C013821282425050405093DF0376
:1025B0004093DE03DF91CF9108956F927F928F92C7
:1025C0009F92AF92BF92CF92DF92EF92FF920F93C2
:1025D0001F93CF93DF938C01009729F4CB010E94C6
:1025E000A8118C01BBC08EEFE82E8FEFF82EE00E05
:1025F000F11E4801860E971E8E149F0408F4ACC08D
:10260000D7014D915C91119746175707B8F04530A7
:10261000510508F4A3C0CA0104978617970708F468
:102620009DC042505040461B570BF40141935193BB
:102630006D937C93CF010E94451290C05B01A41A58
:10264000B50A3801640E751EA091E003B091E10354
:10265000CC24DD24E0E0F0E047C0A615B705A9F5DD
:10266000CD91DC911197CE0102968A159B0568F1F8
:10267000CE018A199B09029612962C9112971396F5
:102680003C91059758F0F40122833383CA19DB0982
:10269000D183C083D7016D937C9309C04E5F5F4F98
:1026A0004C0F5D1FF70151834083C901FC01C11428
:1026B000D10431F0D6011396FC93EE9312974EC0DD
:1026C000F093E103E093E00349C08D919C91119751
:1026D000E817F90708F4FC016D0112968C91129726
:1026E00013969C919C01D901109709F0B6CF809167
:1026F000DE039091DF0386159705E9F4E617F707E7
:10270000D0F420912001309121012115310541F4AF
:102710002DB73EB780911C0190911D01281B390BEC
:1027200082169306C8F49092DF038092DE03F701CD
:102730007183608313C0CB010E94A811EC01009744
:1027400059F0D7014D915C91B8010E949000C801E9
:102750000E9445128E0102C000E010E0C801DF9126
:10276000CF911F910F91FF90EF90DF90CF90BF908E
:10277000AF909F908F907F906F9008950CD0EBC09A
:10278000E3D040F0DAD030F021F45F3F19F0CCC054
:10279000511115C1CFC0F0D098F39923C9F3552337
:1027A000B1F3951B550BBB27AA2762177307840744
:1027B00038F09F5F5F4F220F331F441FAA1FA9F3FA
:1027C00033D00E2E3AF0E0E830D091505040E695EC
:1027D000001CCAF729D0FE2F27D0660F771F881F4D
:1027E000BB1F261737074807AB07B0E809F0BB0B3C
:1027F000802DBF01FF2793585F4F2AF09E3F510560
:1028000068F092C0DCC05F3FECF3983EDCF3869545
:1028100077956795B795F7959F5FC9F7880F911DD5
:102820009695879597F90895E1E0660F771F881FC1
:10283000BB1F621773078407BA0720F0621B730B74
:10284000840BBA0BEE1F88F7E095089504D06894C6
:10285000B111B5C0089598D088F09F5790F0B92F66
:102860009927B751A0F0D1F0660F771F881F991FE5
:102870001AF0BA95C9F712C0B13081F09FD0B1E01B
:1028800008959CC0672F782F8827B85F39F0B93F2B
:10289000CCF3869577956795B395D9F73EF49095E7
:1028A0008095709561957F4F8F4F9F4F0895E89465
:1028B00009C097FB3EF490958095709561957F4F88
:1028C0008F4F9F4F9923A9F0F92F96E9BB27939536
:1028D000F695879577956795B795F111F8CFFAF446
:1028E000BB0F11F460FF1BC06F5F7F4F8F4F9F4F77
:1028F00016C0882311F096E911C0772321F09EE8D5
:10290000872F762F05C0662371F096E8862F70E03A
:1029100060E02AF09A95660F771F881FDAF7880F14
:102920009695879597F9089597F99F6780E870E0E5
:1029300060E008959FEF80EC089500240A94161635
:10294000170618060906089500240A94121613069D
:10295000140605060895092E0394000C11F488232B
:1029600052F0BB0F40F4BF2B11F460FF04C06F5F47
:102970007F4F8F4F9F4F089557FD9058440F551F1D
:1029800059F05F3F71F04795880F97FB991F61F0F1
:102990009F3F79F087950895121613061406551F68
:1029A000F2CF4695F1DF08C0161617061806991FD4
:1029B000F1CF86957105610508940895E894BB27C9
:1029C00066277727CB0197F90895629FD001739FFF
:1029D000F001829FE00DF11D649FE00DF11D929FBB
:1029E000F00D839FF00D749FF00D659FF00D9927FA
:1029F000729FB00DE11DF91F639FB00DE11DF91F1E
:102A0000BD01CF0111240895991B79E004C0991FDD
:102A1000961708F0961B881F7A95C9F78095089538
:102A200097FB092E07260AD077FD04D049D006D09F
:102A300000201AF4709561957F4F0895F6F79095F0
:102A400081959F4F0895A1E21A2EAA1BBB1BFD0181
:102A50000DC0AA1FBB1FEE1FFF1FA217B307E4077D
:102A6000F50720F0A21BB30BE40BF50B661F771FD5
:102A7000881F991F1A9469F76095709580959095B5
:102A80009B01AC01BD01CF01089597FB092E0526DE
:102A90000ED057FD04D0D7DF0AD0001C38F4509573
:102AA0004095309521953F4F4F4F5F4F0895F6F772
:102AB00090958095709561957F4F8F4F9F4F0895AA
:102AC000AA1BBB1B51E107C0AA1FBB1FA617B70754
:102AD00010F0A61BB70B881F991F5A95A9F7809570
:102AE0009095BC01CD010895EE0FFF1F0590F49164
:102AF000E02D099410E0CAECD0E004C0FE010E9471
:0E2B000076152296CC3CD107C9F7F894FFCF8A
:102B0E0030612E30312E313032000E000F001000A9
:102B1E001100120013001400150001FF8000E203E3
:102B2E00000000000000FB03CA0383038C03A10313
:102B3E00B203000000003B0DE30DCE0C020DE20CC3
:022B4E002B0D4D
:00000001FF
